:020000040000FA
:0400000025EF00F0F8
:0200080037D0EF
:0800180085D0036A026EFF0EA1
:100020000226032200D0D8A01200030E016EE70EB4
:1000300002D8F5D7016AFE0F006EE86A015AD8A00F
:1000400012000000000600D0F8D7F86A4F0EAF6E1D
:10005000240EAC6E900EAB6E0001070EB46E0F0E48
:10006000C16EC69AC00E926EE00E936EC00E946E74
:10007000956AE80E966EA8D09EAA1BD0060EAB1409
:1000800012E1E1CF62F0E2CF63F0642A1EEE80F06D
:100090006450E126000EE222AECFE7FF62C0E1FF2E
:1000A00063C0E2FF1100AE50AE50AB98AB881100B8
:1000B0000AD0F2A408D0F2940A4A0B2A817A096A7B
:1000C000D6CF08F0110011006450655C14E0652A79
:1000D000E9CF00F0EACF01F00EEE80F06550E9269E
:1000E000000EEA22EF50006E00C0E9FF01C0EAFFF7
:1000F000D880120004D0E868006ED8A01200120068
:10010000646A656A9D8A9F8AF28EF28C12009D9ABB
:100110000EEE80F0000EEE6AE82EFDD7646A656A86
:100120009D8A1200F29ED8CF5AFEE8CF5BFEE0CF48
:100130005CFEE9CF5DFEEACF5EFEE1CF5FFEE2CF7F
:1001400060FED9CF61FEDACF62FEF6CF63FEF7CF55
:1001500064FEF5CF65FEF3CF66FEF4CF67FEA6CF53
:1001600068FEF28E0001A1925CA207D00E4A0F2A0F
:100170000EA202D00E6A0F6A02D00E6A0F6AF29EB9
:100180005ACED8FF5BCEE8FF5CCEE0FF5DCEE9FF44
:100190005ECEEAFF5FCEE1FF60CEE2FF61CED9FF27
:1001A00062CEDAFF63CEF6FF64CEF7FF65CEF5FFD1
:1001B00066CEF3FF67CEF4FF68CEA6FFF28E100086
:1001C0009EA8FED7AD6E1200939A8A8A140E25DF80
:1001D000939A8A9AAAEC07F05E6A92DF98DFCD6A5A
:1001E000F294F28A870ED56EB16AA192A082B26AA9
:1001F000B36AD08EA292B10EB16E66DF106EB80EE9
:10020000105C09E3FE0E105C03E357EF06F003D029
:10021000126A57EF06F010AE22D0126A870E105CF9
:1002200005E110C012F01368146817D0970E105C27
:1002300005E110C012F0156816680FD0A70E105C0B
:1002400005E110C012F01768186807D0B70E105CEF
:1002500004E110C012F019681A6857EF06F0125244
:1002600004E157EF06F057EF06F0870E125CD8A4B2
:1002700068D0132803E110C013F061D010C014F04F
:10028000400E135C02E1899459D0410E135C02E1E7
:10029000899254D0420E135C02E189904FD0430EF4
:1002A000135C02E189964AD0440E135C02E18998FE
:1002B00045D0450E135C02E1899A40D0460E135C8E
:1002C00002E18D903BD0470E135C02E18D9236D057
:1002D000480E135C02E18D9431D0490E135C02E1AB
:1002E0008A982CD04A0E135C02E18A9627D04B0ED6
:1002F000135C02E18A9422D04C0E135C02E18A92D4
:100300001DD04D0E135C02E18A9018D04E0E135C86
:1003100002E18C9E13D0780E135C02E18B900ED01C
:10032000790E135C02E18B9209D07A0E135C02E124
:100330008B9404D07B0E135CD8B48B96136857EF64
:1003400006F0970E125CD8A447EF06F0152804E1DA
:1003500010C015F046EF06F010C016F01652D8A4E3
:1003600060D0400E155C02E1899459D0410E155CB5
:1003700002E1899254D0420E155C02E189904FD07F
:10038000430E155C02E189964AD0440E155C02E1E9
:10039000899845D0450E155C02E1899A40D0460EF9
:1003A000155C02E18D903BD0470E155C02E18D9209
:1003B00036D0480E155C02E18D9431D0490E155CA3
:1003C00002E18A982CD04A0E155C02E18A9627D069
:1003D0004B0E155C02E18A9422D04C0E155C02E1B2
:1003E0008A921DD04D0E155C02E18A9018D04E0EF7
:1003F000155C02E18C9E13D0780E155C02E18B90A7
:100400000ED0790E155C02E18B9209D07A0E155C44
:1004100002E18B9404D07B0E155CD8B48B9645EF2B
:1004200006F0400E155CD8A443D0D89016365CB0C8
:100430001FD05C80D6CF08F0D7CF09F0540E082427
:10044000046E000E0920056E000E0A20066E000ED6
:100450000B20076E165004241C6E000E05201D6E26
:10046000000E06201E6E000E07201F6E89841ED00F
:100470005C80D6CF08F0D7CF09F0540E0824046E64
:10048000000E0920056E000E0A20066E000E0B20DD
:10049000076E165004241C6E000E05201D6E000E03
:1004A00006201E6E000E07201F6E899445EF06F091
:1004B000410E155CD8A443D0D89016365CB21FD03C
:1004C0005C82D6CF08F0D7CF09F0540E0824046E12
:1004D000000E0920056E000E0A20066E000E0B208D
:1004E000076E16500424206E000E0520216E000EAB
:1004F0000620226E000E0720236E89821ED05C82A9
:10050000D6CF08F0D7CF09F0540E0824046E000EA1
:100510000920056E000E0A20066E000E0B20076EE5
:1005200016500424206E000E0520216E000E0620B9
:10053000226E000E0720236E899245EF06F0420ED0
:10054000155CD8A443D0D89016365CB41FD05C8418
:10055000D6CF08F0D7CF09F0540E0824046E000E51
:100560000920056E000E0A20066E000E0B20076E95
:1005700016500424246E000E0520256E000E062061
:10058000266E000E0720276E89801ED05C84D6CF91
:1005900008F0D7CF09F0540E0824046E000E09208D
:1005A000056E000E0A20066E000E0B20076E165018
:1005B0000424246E000E0520256E000E0620266EF3
:1005C000000E0720276E899045EF06F0430E155C5C
:1005D000D8A443D0D89016365CB61FD05C86D6CF50
:1005E00008F0D7CF09F0540E0824046E000E09203D
:1005F000056E000E0A20066E000E0B20076E1650C8
:100600000424286E000E0520296E000E06202A6E96
:10061000000E07202B6E89861ED05C86D6CF08F090
:10062000D7CF09F0540E0824046E000E0920056E81
:10063000000E0A20066E000E0B20076E16500424D2
:10064000286E000E0520296E000E06202A6E000E70
:1006500007202B6E899645EF06F0440E155CD8A452
:1006600043D0D89016365CB81FD05C88D6CF08F03F
:10067000D7CF09F0540E0824046E000E0920056E31
:10068000000E0A20066E000E0B20076E1650042482
:100690002C6E000E05202D6E000E06202E6E000E14
:1006A00007202F6E89881ED05C88D6CF08F0D7CF60
:1006B00009F0540E0824046E000E0920056E000E89
:1006C0000A20066E000E0B20076E165004242C6EB6
:1006D000000E05202D6E000E06202E6E000E072047
:1006E0002F6E899845EF06F0450E155CD8A443D0CF
:1006F000D89016365CBA1FD05C8AD6CF08F0D7CF18
:1007000009F0540E0824046E000E0920056E000E38
:100710000A20066E000E0B20076E16500424306E61
:10072000000E0520316E000E0620326E000E0720EE
:10073000336E898A1ED05C8AD6CF08F0D7CF09F0F5
:10074000540E0824046E000E0920056E000E0A20C7
:10075000066E000E0B20076E16500424306E000E3D
:100760000520316E000E0620326E000E0720336E1B
:10077000899A45EF06F0460E155CD8A443D0D89070
:1007800016365CBC1FD05C8CD6CF08F0D7CF09F0F2
:10079000540E0824046E000E0920056E000E0A2077
:1007A000066E000E0B20076E16500424346E000EE9
:1007B0000520356E000E0620366E000E0720376EBF
:1007C0008D801ED05C8CD6CF08F0D7CF09F0540EA8
:1007D0000824046E000E0920056E000E0A20066E25
:1007E000000E0B20076E16500424346E000E0520F8
:1007F000356E000E0620366E000E0720376E8D9087
:1008000045EF06F0470E155CD8A442D0D8901636B6
:100810005CBE1FD05C8ED6CF08F0D7CF09F0540E47
:100820000824046E000E0920056E000E0A20066ED4
:10083000000E0B20076E16500424386E000E0520A3
:10084000396E000E06203A6E000E07203B6E8D8238
:100850001ED05C8ED6CF08F0D7CF09F0540E0824F6
:10086000046E000E0920056E000E0A20066E000EB2
:100870000B20076E16500424386E000E0520396ECA
:10088000000E06203A6E000E07203B6E8D92FDD1C1
:10089000480E155CD8A442D0D89016365DB01FD053
:1008A0005D80D6CF08F0D7CF09F0540E0824046E2F
:1008B000000E0920056E000E0A20066E000E0B20A9
:1008C000076E165004243C6E000E05203D6E000E8F
:1008D00006203E6E000E07203F6E8D841ED05D8088
:1008E000D6CF08F0D7CF09F0540E0824046E000EBE
:1008F0000920056E000E0A20066E000E0B20076E02
:10090000165004243C6E000E05203D6E000E06209D
:100910003E6E000E07203F6E8D94B7D1490E155CD8
:10092000D8A442D0D89016365DB21FD05D82D6CF03
:1009300008F0D7CF09F0540E0824046E000E0920E9
:10094000056E000E0A20066E000E0B20076E165074
:100950000424406E000E0520416E000E0620426EFB
:10096000000E0720436E8A881ED05D82D6CF08F025
:10097000D7CF09F0540E0824046E000E0920056E2E
:10098000000E0A20066E000E0B20076E165004247F
:10099000406E000E0520416E000E0620426E000ED5
:1009A0000720436E8A9871D14A0E155CD8A442D0B4
:1009B000D89016365DB41FD05D84D6CF08F0D7CF5F
:1009C00009F0540E0824046E000E0920056E000E76
:1009D0000A20066E000E0B20076E16500424446E8B
:1009E000000E0520456E000E0620466E000E072004
:1009F000476E8A861ED05D84D6CF08F0D7CF09F027
:100A0000540E0824046E000E0920056E000E0A2004
:100A1000066E000E0B20076E16500424446E000E66
:100A20000520456E000E0620466E000E0720476E1C
:100A30008A962BD14B0E155CD8A442D0D89016368E
:100A40005DB61FD05D86D6CF08F0D7CF09F0540E23
:100A50000824046E000E0920056E000E0A20066EA2
:100A6000000E0B20076E16500424486E000E052061
:100A7000496E000E06204A6E000E07204B6E8A84D7
:100A80001ED05D86D6CF08F0D7CF09F0540E0824CB
:100A9000046E000E0920056E000E0A20066E000E80
:100AA0000B20076E16500424486E000E0520496E78
:100AB000000E06204A6E000E07204B6E8A94E5D089
:100AC0004C0E155CD8A442D0D89016365DB81FD015
:100AD0005D88D6CF08F0D7CF09F0540E0824046EF5
:100AE000000E0920056E000E0A20066E000E0B2077
:100AF000076E165004244C6E000E05204D6E000E3D
:100B000006204E6E000E07204F6E8A821ED05D8832
:100B1000D6CF08F0D7CF09F0540E0824046E000E8B
:100B20000920056E000E0A20066E000E0B20076ECF
:100B3000165004244C6E000E05204D6E000E06204B
:100B40004E6E000E07204F6E8A929FD04D0E155CA0
:100B5000D8A442D0D89016365DBA1FD05D8AD6CFC1
:100B600008F0D7CF09F0540E0824046E000E0920B7
:100B7000056E000E0A20066E000E0B20076E165042
:100B80000424506E000E0520516E000E0620526E99
:100B9000000E0720536E8A801ED05D8AD6CF08F0E3
:100BA000D7CF09F0540E0824046E000E0920056EFC
:100BB000000E0A20066E000E0B20076E165004244D
:100BC000506E000E0520516E000E0620526E000E73
:100BD0000720536E8A9059D04E0E155CD8A442D08F
:100BE000D89016365DBC1FD05D8CD6CF08F0D7CF1D
:100BF00009F0540E0824046E000E0920056E000E44
:100C00000A20066E000E0B20076E16500424546E48
:100C1000000E0520556E000E0620566E000E0720B1
:100C2000576E8C8E1ED05D8CD6CF08F0D7CF09F0D2
:100C3000540E0824046E000E0920056E000E0A20D2
:100C4000066E000E0B20076E16500424546E000E24
:100C50000520556E000E0620566E000E0720576EBA
:100C60008C9E13D0780E155C02E18B800ED0790E2D
:100C7000155C02E18B8209D07A0E155C02E18B844F
:100C800004D07B0E155CD8B48B86156810D0A70EE7
:100C9000125C02E10CD00BD0B70E125C08E11928EF
:100CA00003E110C019F003D010C01AF043D95C5210
:100CB000D8B4A8D05CA013D0D6CF08F0D7CF09F015
:100CC0001C50085C1D5009581E500A581F500B58E4
:100CD0000B501F18D8B0800A02E789945C905CA280
:100CE00013D0D6CF08F0D7CF09F02050085C2150A0
:100CF000095822500A5823500B580B502318D8B0CB
:100D0000800A02E789925C925CA413D0D6CF08F0E7
:100D1000D7CF09F02450085C2550095826500A58AE
:100D200027500B580B502718D8B0800A02E789903B
:100D30005C945CA613D0D6CF08F0D7CF09F028502A
:100D4000085C295009582A500A582B500B580B5050
:100D50002B18D8B0800A02E789965C965CA813D05D
:100D6000D6CF08F0D7CF09F02C50085C2D50095889
:100D70002E500A582F500B580B502F18D8B0800AFD
:100D800002E789985C985CAA13D0D6CF08F0D7CF39
:100D900009F03050085C3150095832500A5833502D
:100DA0000B580B503318D8B0800A02E7899A5C9A26
:100DB0005CAC13D0D6CF08F0D7CF09F03450085C24
:100DC0003550095836500A5837500B580B503718C1
:100DD000D8B0800A02E78D905C9C5CAE13D0D6CF71
:100DE00008F0D7CF09F03850085C395009583A500C
:100DF0000A583B500B580B503B18D8B0800A02E7FA
:100E00008D925C9E5D52D8B493D05DA013D0D6CFA6
:100E100008F0D7CF09F03C50085C3D5009583E50CF
:100E20000A583F500B580B503F18D8B0800A02E7C1
:100E30008D945D905DA213D0D6CF08F0D7CF09F086
:100E40004050085C4150095842500A5843500B58D2
:100E50000B504318D8B0800A02E78A985D925DA4CF
:100E600013D0D6CF08F0D7CF09F04450085C4550D6
:100E7000095846500A5847500B580B504718D8B0DD
:100E8000800A02E78A965D945DA613D0D6CF08F05B
:100E9000D7CF09F04850085C495009584A500A58C1
:100EA0004B500B580B504B18D8B0800A02E78A946D
:100EB0005D965DA813D0D6CF08F0D7CF09F04C507F
:100EC000085C4D5009584E500A584F500B580B5063
:100ED0004F18D8B0800A02E78A925D985DAA13D0B5
:100EE000D6CF08F0D7CF09F05050085C51500958C0
:100EF00052500A5853500B580B505318D8B0800A10
:100F000002E78A905D9A5DAC13D0D6CF08F0D7CFB8
:100F100009F05450085C5550095856500A5857501B
:100F20000B580B505718D8B0800A02E78C9E5D9C76
:100F3000FDEF00F0420E195C07E11A5203E15E90EA
:100F400009D801D05E8004D07B0E195CD8B402D8D9
:100F5000196812005C6A5D6A0A6A0B6A8994899250
:100F6000899089968998899A8D908D928D948A9886
:100F70008A968A948A928A908C9E8B908B928B947C
:060F80008B961200FFD762
:020000040030CA
:0300010006160ED2
:020005008580F4
:060008000FC00FE00F40E5
:00000001FF
